:020000040000FA
:020000000B28CB
:0800080005280130851DFF30C1
:10001000A8078B101B2883169F01403081000430F5
:100020009500CC30850061308F0083120730990035
:100030002B2090308B002008850036203B20A0012B
:10004000261C2014231CA014241CA016033073208B
:10005000843067201B28A701A601A501A401A301E4
:10006000A201A1012330A000A801080028088316DE
:10007000900083120800A70A0A3027020319A7017B
:100080000319A60A0A3026020319A6010319A50AB4
:100090000A3025020319A50103198B170319A40AB5
:1000A0000A3024020319A4010319A30A0A30230207
:1000B0000319A3010319A20A0A3022020319A2019B
:1000C0000319A10A0A3021020319A1010800F13E17
:1000D000A90029186B28A9186D28A9186F28FC3EBB
:1000E00003186F280800FF3EAA005E3067206030CA
:1000F0006720AA0B77280800FF3EAB00633073200F
:100100005D306720633073205F306720AB0B82283F
:1001100008008D208E208E208D208E2091200000C2
:0401200000000800D3
:02400E00D537A4
:00000001FF
